:020000040000FA
:100000000A128A11C82A8A002808093E03188A0A97
:1000100082000034003400340034003400340034F2
:100020002F340034003400340734003407340034F3
:1000300014347F3414347F34143424342A347F3419
:100040002A341234C434C834103426344634363496
:1000500049345534223450340034053403340034E8
:10006000003400341C342234413400340034413430
:1000700022341C340034143408343E34083414342C
:10008000083408343E340834083400340034503422
:100090003034003410341034103410341034003440
:1000A00060346034003400342034103408340434B4
:1000B00002343E345134493445343E340034423401
:1000C0007F3440340034423461345134493446344E
:1000D0002134413445344B3431341834143412341F
:1000E0007F341034273445344534453439343C3476
:1000F0004A344934493430340134713409340534D4
:1001000003343634493449344934363406344934B6
:10011000493429341E340034363436340034003443
:100120000034563436340034003408341434223465
:10013000413400341434143414341434143400347A
:100140004134223414340834023401345134093433
:10015000063432344934593451343E347E34113407
:10016000113411347E347F344934493449343634BF
:100170003E3441344134413422347F3441344134BB
:1001800022341C347F3449344934493441347F3477
:1001900009340934093401343E3441344934493492
:1001A0007A347F340834083408347F3400344134DE
:1001B0007F34413400342034403441343F340134FE
:1001C0007F3408341434223441347F344034403492
:1001D000403440347F3402340C3402347F347F3472
:1001E0000434083410347F343E34413441344134D3
:1001F0003E347F3409340934093406343E34413402
:10020000513421345E347F3409341934293446346E
:1002100046344934493449343134013401347F346B
:10022000013401343F344034403440343F341F34CF
:100230002034403420341F343F3440343834403488
:100240003F346334143408341434633407340834CA
:1002500070340834073461345134493445344334FC
:1002600000347F3441344134003455342A34553419
:100270002A3455340034413441347F34003404345A
:1002800002340134023404344034403440344034C5
:100290004034003401340234043400342034543403
:1002A0005434543478347F34483444344434383407
:1002B00038344434443444342034383444344434BA
:1002C00048347F3438345434543454341834083473
:1002D0007E340934013402340C34523452345234F2
:1002E0003E347F34083404340434783400344434E5
:1002F0007D34403400342034403444343D340034C0
:100300007F341034283444340034003441347F3492
:10031000403400347C3404341834043478347C346D
:1003200008340434043478343834443444344434A1
:1003300038347C3414341434143408340834143409
:10034000143418347C347C340834043404340834D1
:100350004834543454345434203404343F34443412
:10036000403420343C344034403420347C341C3419
:100370002034403420341C343C3440343034403455
:100380003C34443428341034283444340C3450344D
:10039000503450343C344434643454344C34443455
:1003A000820720342A3420344534523441345334C3
:1003B0004534203445344534503452344F344D3470
:1003C00020344D3445344D344F3452345934203474
:1003D0002A34203482072A342034353420346B34D4
:1003E000573420342A3482072A3432342E343534B8
:0803F00020346B3457342A3429
:10040000820749344E3420342034203420342034C0
:10041000203420342034203420342034203420343C
:10042000203420344F345534543420342034203494
:10043000203420348207503452344F3447345234FD
:1004400041344D342034623461347334653464345F
:1004500020346F346E3420344A3441344C344C34BC
:1004600049344234203482072A342A342A342A3444
:10047000203453344D3441345234543420344D34C8
:10048000453454344534523420342A342A342A34FE
:100490002A342A342A342A3482072A342A342A3441
:1004A0002A342A342A342034483461346E347A347D
:1004B00065346D3461346E3420342A342A342A345D
:1004C0002A342A34383465342A34820720344F34AD
:1004D0005534543482074F346D3461347834820794
:1004E00049346D34613478348207203449344E34D1
:1004F0002E34820720344E3472342E341030A8004B
:100500000310A40DA50D0310A00DA10D031C8E2A30
:100510002308A5072208A4070318A50AA80B802A08
:1005200008001030A800A201A3010310A60DA70D1A
:100530000310A00DA10DA20DA30D23082502031D7C
:10054000A32A220824020319A72A0318AE2A250881
:10055000A3022408A202031CA3032614A80B952AB5
:100560000800AB1BC22A2B1BBD2A2A088400831358
:10057000AB08031D8317000808002A08A9002B08F0
:100580003F39C32A08008A00831203132A08820015
:100590009F01073083169F0007309C000E2B81308F
:1005A0008316990018150800980183129801CF222C
:1005B000831603138C120C128717071798168312D1
:1005C00098171816080083160317D4008312031314
:1005D0000C1AEB2AE62A8316031754088312031316
:1005E00099000800831203138C1EFE2A1A08831632
:1005F0000317D200831203138C12022B83160317E6
:100600005310092B981C062B181218168316031763
:10061000531453180C2BF22A52080800D4228316C4
:10062000031307118312AC010130AD008A110A12C5
:100630004B2B83160317D10083120313AC01013037
:10064000AD002C0383169200013003175102031DE5
:100650002F2BFC308312031392051215080004306F
:100660005102031D3B2BFC3083120313120501388A
:1006700092001215080010305102031D472BFC3068
:100680008312031312050238920012150800831218
:10069000031312110800D201D3010B2CF030831286
:1006A000031353050C38D3005208950053089700E4
:1006B000080003305002031D5F2BFF304F02031967
:1006C000672B031C672BFF30CF000330D0000310D3
:1006D000500C83120313A100831603174F0C8312CF
:1006E0000313A0000310A10CA00C2008D2000330BB
:1006F000831603174F0583120313A000200EA100D9
:100700003030A105CF3053052104D3004E2B831682
:100710000317C6004608031D902BC701C801FC2B18
:10072000643046020319962B031CA62B8312031375
:100730002D0883160317C800831203132C03831696
:100740000317C700470A0319C803FC2B4608C90052
:10075000CA010310831203132D0C83160317CC0058
:10076000831203132C0C83160317CB000310CC0C3D
:10077000CB0C490883120313A000831603174A0801
:1007800083120313A100831603174B08831203136C
:10079000A200831603174C0883120313A3007E22C2
:1007A00083120313240883160317CD008312031347
:1007B000250883160317CE00193083120313A400F3
:1007C000A501831603174D0883120313A000831697
:1007D00003174E0883120313A1008A110A129122F3
:1007E00083120313260883160317C700831203130B
:1007F000270883160317C8000310470DC900480DCA
:10080000CA000310C90DCA0D4908CF004A08D0001C
:100810008A110A12592B013019238A110A124E2308
:1008200032308A110A128723831603130516051422
:10083000851405158A110A126F2D420883128D0046
:100840008316430883128F0083168C170C14000044
:10085000000083120C088316C40083120E0883164E
:10086000C50008003E08C2003F08C3001D248316CF
:1008700003174408C0004508C10040088312031351
:10088000A00083160317410883120313A100080078
:100890003D108B1B3D14FC302A05AE002B08AF0029
:1008A000B8010310380DB9002F08BB0038082E0717
:1008B000BA000318BB0A3A08BE003B08BF00322446
:1008C000B03083160317390784008317831203138C
:1008D00020088000840A2108800083160317B80AC4
:1008E000043038028A110A12031D512C03302A05E4
:1008F000B900BA010310390DBB003A0DBC00B0308D
:100900003B07840083172C088000840A2D08800090
:100910002E0883128D0083162F0883128F008316F2
:10092000B8010310380DB900B030390784008317BF
:100930000008AC00840A0008AD002C0883128C006B
:1009400083162D0883128E0083168C170C158B13BB
:1009500055308D00AA308D008C14000000000C1161
:1009600083128D0A8316B80A04303802031D912CB5
:100970003D18BC2C8B1308008B1708002408A60018
:100980002508A700A801A901D92C8312031306305A
:10099000A000A530A1000A128A11A10BCB2C0A12CB
:1009A0008A11A00BC92C000083160317A80A03198B
:1009B000A90A2808260283120313A000831603172E
:1009C00029082702831203132004031DC52C0800E5
:1009D0001E08A0001F08A100A201A301092D831277
:1009E00003135E30A000FD30A1000330A2000A1204
:1009F0008A11A20BF72C0A128A11A10BF52C0A12EC
:100A00008A11A00BF32C000083160317A20A031906
:100A1000A30A2208200283120313A00083160317DF
:100A200023082102831203132004031DEF2C080066
:100A30001508990016089A0019089C001A089D00CC
:100A40009B01442D83160317180883120313AB0070
:100A5000831603171B08170783120313AA00031832
:100A6000AB0AB12283120313A000831603171308E5
:100A700083120313AA008316031714088A110A129B
:100A8000C322831603179B0A1B081C02831203133D
:100A9000A000831603171D088312031320048A1174
:100AA0000A12031D222D08000317920001301202C2
:100AB000031D602D013083120313D4000530D500CF
:100AC000831603171208FF30120208000130540287
:100AD000031D6E2D4D08A8004E0803280034013078
:100AE000542583120313D6010130D7008A150A1248
:100AF000512983120313C900CF124F08860000004A
:100B000000000000000000004A188A2DCF144F0892
:100B100086008D2D4F144F0886004F114F08860018
:100B2000000000000000000000004908D10051084A
:100B30008800831688018312CF164F0886000000B4
:100B400000000000000000000000000000000000A5
:100B50000000CF124F0886000000000000000000D7
:100B60000000CF104F0886004F104F088600080085
:100B7000CF124F08860000000000000000000000B7
:100B80004C18C62DCF144F088600C92D4F144F089E
:100B900086004F154F08860000000000000000008E
:100BA0000000CF164F088600000000000000000083
:100BB000000000000000000000000000CF124F08FD
:100BC000860000000000000000000000FF308316D7
:100BD000880083120808CB00CF104F0886004F1002
:100BE0004F0886004B080800831203134A103F3059
:100BF0007925831203134A143F308A110A12792D82
:100C0000E1006910403061020319082E031C0B2E0D
:100C10004030E102691403134F124F0886003F3041
:100C200003176105EA0040306A04EB0069181B2EC7
:100C300003134A101D2E03134A1403176B0879255A
:100C4000031083120317620CE7000310E70C031074
:100C5000E70C07306705EC00B8306C04ED008A1132
:100C60000A126918362E03134A10382E03134A1439
:100C700003176D087925831203134F164F0886005A
:100C800003178A110A126918482E03134C104A2EB2
:100C900003134C14B82583120317E3008A110A12B8
:100CA0006918552E03134C10572E03134C14B825F6
:100CB00083120317E3000130031357028A110A124B
:100CC000031D742E073003176205E4006408FE005C
:100CD0000130E5007E086F2E0310E50DFE03031DB5
:100CE0006C2E6508E304872E073003176205E400C5
:100CF0006408FE000130E5007E08812E0310E50D3A
:100D0000FE03031D7E2E6509E6006608E305031356
:100D10004F124F0886003F3003176105EE00403048
:100D20006E04EF006918972E03134A10992E0313CF
:100D30004A1403176F087925031083120317620CF6
:100D4000E8000310E80C0310E80C07306805831670
:100D50009000B8301004910083128A110A126918A9
:100D6000B42E03134A10B62E03134A148316031726
:100D700011087925831203134F164F0886000317B5
:100D80008A110A126918C72E03134A10C92E0313B9
:100D90004A1403176308792DBA00411040303A0213
:100DA0000319D42E031CD72E4030BA0241144F121F
:100DB0004F0886003F303A05C20040304204C3006D
:100DC0004A1041184A14430879250310831203136B
:100DD0003B0CC0000310C00C0310C00C07304005D2
:100DE000C200B8304204C3004A1041184A144308F4
:100DF0008A110A127925831203134F164F088600B1
:100E000007303B05BD003D088A110A12031D0D2F56
:100E10004A1041184A143C08792D4C1041184C14C2
:100E2000B82583120313C2004C1041184C148A11C8
:100E30000A12B82583120313C20007303B05BD0018
:100E40003D09BE000930BE073E08FE00FF30BF006E
:100E5000FE088A110A120319312F0310BF0CFE0B72
:100E60002D2F3F08C20507303B05BD003D08FE00A1
:100E70003C08BE007E083F2F0310BE0DFE03031D7D
:100E80003C2F3E08C2044F124F0886003F303A05FF
:100E9000C60040304604C7004A1041184A144708AB
:100EA00079250310831203133B0CC3000310C30CFA
:100EB0000310C30C07304305C600B8304604C70012
:100EC0004A1041184A1447088A110A1279258312D8
:100ED00003134F164F0886004A1041184A1442085F
:100EE0008A110A127925831203134F124F088600C4
:100EF0003F303A05C60040304604C7004A1041184A
:100F00004A1447088A110A12792503108312031321
:100F10003B0CBD000310BD0C0310BD0C3D0AC4000A
:100F200007304405C600B8304604C7004A104118CF
:100F30004A1447088A110A127925831203134F169F
:100F40004F0886004C1041184C148A110A12B8251B
:100F500083120313C2004C1041184C148A110A1258
:100F6000B82583120313C20007303B05BD003D08BE
:100F7000FE00FF30BE007E088A110A12C22F031045
:100F8000BE0DFE03031DBF2F3E08C20507303B0503
:100F9000BD003D09BE000930BE073E08FE003C080A
:100FA000BF00FE080319D82F0310BF0CFE0BD42F6F
:100FB0003F08C2044F124F0886003F303A05C60072
:100FC00040304604C7004A1041184A1447087925A2
:100FD0000310831203133B0CBD000310BD0C031060
:100FE000BD0C3D0AC50007304505C600B8304604B3
:100FF000C7004A1041184A1447088A110A12792575
:10100000831203134F164F0886004A1041184A14E2
:1010100042088A110A12792D0317D400D50103134F
:101020004F124F088600073003175505D700B83018
:101030005704D80003134A10031758088A1179255A
:101040000730831203175505D900B8305904DA0068
:1010500003134A1403175A088A110A1279258312B6
:101060000317DB013F305B05DC0040305C04DD0032
:1010700003134A1003175D088A110A127925831297
:101080000317DE013F305E05DF0040305F04E00003
:1010900003134A14031760088A110A127925831270
:1010A00003134F164F0886000317D60103134A1087
:1010B000031754088A110A127925831203134A145C
:1010C000031754088A110A12792583120317D60AC6
:1010D000803056028A150A12031D5628D50A083098
:1010E0005502031D0F2808008312031350105008E7
:1010F0008700000000000000000000000000000069
:101100000000000000005014500887005608031D1E
:101110008E2800300C208A150A129028FF300C20EF
:10112000831203134F124F0886000317C8010730BC
:101130004805C900B8304904CA0003134A10031710
:101140004A088A110A12792583120317CB01073046
:101150004B05CC00B8304C04CD0003134A140317E0
:101160004D088A110A12792583120317CE013F30E8
:101170004E05CF0040304F04D00003134A10031730
:1011800050088A110A12792583120317D1013F30C2
:101190005105D20040305204D30003134A14031700
:1011A00053088A110A1279258A110A12F42DD101E5
:1011B000510888008316880183124F164F08860055
:1011C0004F114F088600CF164F088600CF104F08EA
:1011D00086004F104F088600501450088700831671
:1011E0000611061286128610061007107428AF002A
:1011F0002030310239100319FF28031C39147A30CA
:101200003102B910031906290318B9143911391C10
:10121000B9183915391D0E292030B100203031029E
:10122000B500B6015508A000A1013508A200360896
:10123000A3008A117E22831203132408B20025081A
:10124000B3005508B700B8018A150A124A29803040
:101250002F0203192D29031C2E2908003208CD0066
:101260003308CE008A11662583120313B400570891
:101270008A150A120319B4093008BB003408BC00EF
:101280002F088A11CC2683120313B20A0319B30A5A
:10129000AF0AB80A380837028A150A12031D27292F
:1012A0000800D801D9018A2A831203132008AE004E
:1012B0005908B0002E08B10058088A150A12F72004
:1012C000831203135508D807080083120317AA00D6
:1012D0002C08AE00AF012A08B000B10131082F027E
:1012E000B30030082E02B200031CB3032D08AE0079
:1012F000AF012B08B000B10131082F02B500300852
:101300002E02B400031CB5030310320DB600330DDA
:10131000B7000310340DB800350DB9002A08BA0023
:10132000BB012B08BC00BD010130BE00BF01013074
:10133000C000C1013308803A0313A00080302002AE
:10134000031DA5290030031732020319B72903181A
:10135000B729FF300317BE00BF00B209B309B20AB4
:101360000319B30AB609B709B60A0319B70A03176E
:101370003508803A0313A00080302002031DC329E2
:101380000030031734020319D5290318D529FF307B
:101390000317C000C100B409B509B40A0319B50A9E
:1013A000B809B909B80A0319B90A03172B08E200EA
:1013B0002A088A11002683120317320833044615BF
:1013C0000319461134083504C6150319C61146120F
:1013D000461DC61946168A150A12461E892A330862
:1013E000803A0313A00003173508803A0313200244
:1013F000031DFD290317340832020319012A031CB7
:10140000452A0317C201C301831203173A082C02AD
:101410000313A00003173B08031320040319892AB0
:1014200003173F08BB073E08BA070318BB0A390871
:10143000C3073808C2070318C30A3308803A0313E6
:10144000A00003174308803A03132002031D2B2A30
:1014500003174208320203193C2A03183C2A0317D7
:101460004108BD074008BC070318BD0A3708C3027E
:101470003608C202031CC30303173C08E2003A0803
:101480008A1100268A150A12042A0317C401C5010D
:10149000831203173C082D020313A00003173D0815
:1014A000031320040319892A03174108BD074008C4
:1014B000BC070318BD0A3708C5073608C407031858
:1014C000C50A3508803A0313A00003174508803A7F
:1014D00003132002031D6F2A031744083402031963
:1014E000802A0318802A03173F08BB073E08BA0763
:1014F0000318BB0A3908C5023808C402031CC50317
:1015000003173C08E2003A088A1100268A150A12DD
:10151000482A0800D720303083120313DA00313014
:10152000DB003230DC003330DD002E30DE003430C2
:10153000DF003530E0003030E1003630E20032309C
:10154000E3003130E4002E30E5003830E60036307C
:10155000E700EE01EF018316A401A501A601A70192
:10156000A801A901AA018312D60105308316AF0094
:101570000530B0000530B1008A110A162F2C7420F6
:10158000013083120313D7008316A801A901831623
:1015900028088312A000831629088312A1000A30AC
:1015A000A200A3018A110A127E22831203132408C7
:1015B0000317A000031325080317A1002108A300A7
:1015C00004302007A2000318A30A83160313280877
:1015D0008312A000831629088312A1000A30A200FA
:1015E000A3018A110A127E2283120313240803170F
:1015F000A400031325080317A5002508A70004303D
:101600002407A6000318A70A1830AB002608AC0070
:101610001A30AD0022088A150A12652183160313B9
:10162000A80A0319A90A0D3028028312A00000306D
:1016300083162902831220048A150A12031DC72A61
:1016400032300317AB007E30AC00AD017E30652137
:1016500083160313A801A901831628088312A0008A
:10166000831629088312A1000530A200A3018A1164
:101670000A127E228312031324080317A000031307
:1016800025080317A1008316031328088312A0005E
:10169000831629088312A1000530A200A3018A1134
:1016A0000A127E228312031324080317A2000313D5
:1016B00025080317A3002008AB007E30AC002208E9
:1016C000AD007C308A150A12652183160313A80A1F
:1016D0000319A90A0B3028028312A00000308316D8
:1016E0002902831220048A150A12031D2C2B0130B3
:1016F0008316A800A90183120317A8013730A90097
:1017000028080313D800031729080313D9005430FD
:101710008316031793000930940019309500960141
:10172000013097000230403898008A1118250130A6
:10173000831603179E009F018A110A12E82C8A1152
:10174000F22283120313E8007F30E80508008312B9
:1017500003179701980103136C086D0403171F14F6
:10176000031D1F1003136A086B0403179F1403194A
:101770009F101F151F189F1C1F1103136C086D0469
:1017800003179F1503199F1103136A086B040317AE
:101790001F16031D1F129F169F191F1E9F121F1336
:1017A0001F1D9F1A1F171F1F0F2C0A300313A400A1
:1017B000A5016C08A0006D08A1008A119122831276
:1017C00003132608031799000313270803179A0029
:1017D0001A089C00323019079B0003189C0A0A3033
:1017E0000313A400A5016A08A0006B08A1008A11D8
:1017F0000A12912283120313260803179D00031374
:10180000270803179E001E081C0298001D081B02D3
:101810009700031C980317088A110A12872B0800E7
:1018200096000530E20016088A110026831203177D
:10183000AB011608AC000330AD0016088A150A1279
:101840006529013083120313D7008316A801A9016B
:10185000EF01290883120317910083160313280848
:101860002A078312031790000318910AF03003131C
:10187000A400A501031710080313A0000317110803
:101880000313A1008A1191228312031322088316E5
:10189000AB00831223088316AC001B30AC07583012
:1018A000AB070318AC0A2B080317BE0003132C0860
:1018B0000317BF008A110A1232248312031320086F
:1018C0008316AD00831221088316AE002F08831201
:1018D000A400A50183162D088312A00083162E08EC
:1018E0008312A1008A110A1291228312031326087F
:1018F0008316AD00831227088316AE0000302E0237
:101900008A150A12031D862C32302D0203198C2CE5
:10191000031C8C2CAD01AE0100302E02031D922C55
:101920001C302D020319A92C031CA92C1930AD0061
:10193000AE012809831203179000831603132909A7
:101940008312031791007D3090070318910A100845
:10195000102483160313280983120317900083169B
:10196000031329098312031791007D309007031890
:10197000910A831603132E0883120317930019305C
:10198000831603132D078312031792000318930A7B
:101990008316031328098312031794008316031375
:1019A00029098312031795007D3094070318950ABF
:1019B0001208AB001408AC001930AD0010088A15ED
:1019C0000A126521013083160313AC07E030AB0720
:1019D0000318AC0A2B080317BE0003132C080317C7
:1019E000BF008A110A1232248312031320088316BF
:1019F000AD00831221088316AE002F088312A400C5
:101A0000A50183162D088312A00083162E088312C9
:101A1000A1008A110A129122831203132608831649
:101A2000AD00831227088316AE0000302E028A15FF
:101A30000A12031D1D2D19302D020319332D031C0D
:101A4000332DAD01AE0128098312031790008316D0
:101A5000031329098312031791007D30900703189F
:101A6000910A100810248316031328098312031700
:101A700090008316031329098312031791007D3008
:101A800090070318910A831603132D098312031775
:101A90009200831603132E098312031793001A3042
:101AA00092070318930A8316031328098312031756
:101AB00094008316031329098312031795007D30C0
:101AC00094070318950A1208AB001408AC001930EB
:101AD000AD0010088A150A12652183160313A80A9F
:101AE0000319A90AEF0A78306F028A150A12031D3A
:101AF000292C080083125D088316E10083125E081A
:101B00008316E20083125F088316E30083126008E5
:101B10008316E4000F30E9003730EA0069088312C9
:101B2000D80083166A088312D9005430831603172D
:101B3000930009309400043095009601E13097003D
:101B400098018A1118258312031364088316E5008F
:101B5000831265088316E600831266088316E70081
:101B6000831267088316E8006930EB003730EC0019
:101B70006B088312D80083166C088312D900543086
:101B800083160317930009309400043095009601E2
:101B9000E530970098018A110A121825283083161B
:101BA0000313ED003730EE006D088312D800831662
:101BB0006E088312D9008A150A128518F42D053093
:101BC0008316AF0054300317930009309400083097
:101BD00095009601F43097000130403898008A1142
:101BE00018258A150A12062E0A308316AF005430C3
:101BF0000317930009309400083095009601EB30EC
:101C000097000130403898008A1118258316031375
:101C10002F0830028A150A120319142E2F08B0005B
:101C2000BF228A150A122124831203138A150A126D
:101C300005191E2E23308316B100080005308316C7
:101C4000B1000800573083160317C2001B30C300D1
:101C50008A111D248316031744080313AA002A08B7
:101C60006014031D6010EF302A02E0108A150A127A
:101C700003193C2E0318E0146011601CE018601575
:101C8000601D452EEF30AA00462EAA0357300317D9
:101C9000AA001B30AB0003132A080317AC00AD01E8
:101CA0008A114824031083160313A50CA40C0030DA
:101CB00025028A150A12031D5F2EFF302402031924
:101CC000662E031C662EFF30A400A5010310A70C8E
:101CD000A60C00302702031D6F2EFF3026020319C9
:101CE000762E031C762EFF30A600A70183126E0805
:101CF000A4006F08A500831620088312A000831695
:101D000021088312A1008A1191228312031326084D
:101D10008316DE00831227088316DF0003105F0C92
:101D2000A1005E0CA000003021028A150A12031DDA
:101D30009B2EFF3020020319A22E031CA22EFF307F
:101D4000A000A10183126E08A4006F08A5008316ED
:101D500022088312A000831623088312A1008A118F
:101D600091228312031326088316DE0083122708AC
:101D70008316DF0003105F0CA3005E0CA20000308E
:101D800023028A150A12031DC72EFF3022020319EF
:101D9000CE2E031CCE2EFF30A200A3011B30AC00C0
:101DA00058302A07AB000318AC0A2B080317AA0007
:101DB00003132C080317AB00031320080317AC0010
:101DC000031321080317AD008A114824F03083164D
:101DD0000313AB070318AC0A2B080317AA0003135D
:101DE0002C080317AB00031324080317AC000313DC
:101DF00025080317AD008A110A124824F030831613
:101E00000313AB070318AC0A2B080317AA0003132C
:101E10002C080317AB00031322080317AC000313AD
:101E200023080317AD008A110A124824F0308316E4
:101E30000313AB070318AC0A2B080317AA000313FC
:101E40002C080317AB00031326080317AC00031379
:101E500027080317AD008A110A1248248A150A12AE
:101E6000BF228A150A12212483120313EE01EF0107
:101E70008316A001A101A201A3018312EA01EB01D3
:101E8000EC01ED018316A401A501A601A70108003C
:101E9000573083160317C2001B30C3008A111D245C
:101EA0008316031744080313AA00CF01D001D10100
:101EB00002308A004F088A110A124C228A110A1233
:101EC000E32283160313CF0A0319D00AD10A103074
:101ED00051028A150A12031D582F0D308A11E32270
:101EE0000A308A110A12E32283160313CF01D001AC
:101EF000D80102308A004F088A110A1279228A1109
:101F00000A12E32283160313CF0A0319D00AD80A50
:101F1000043058028A150A12031D792F09308A11DC
:101F2000E32283160313CF01D001D90102308A00C6
:101F30004F088A110A1274228A110A12E3228316A8
:101F40000313CF0A0319D00AD90A043059028A159B
:101F50000A12031D962F09308A11E32283160313F8
:101F6000CF01D001DA0102308A004F088A110A122B
:101F70006F228A110A12E32283160313CF0A031970
:101F8000D00ADA0A04305A028A150A12031DB32F46
:101F900009308A11E32283160313CF01D001DB013C
:101FA00002308A004F088A110A1265228A110A1229
:101FB000E32283160313CF0A0319D00ADB0A043085
:101FC0005B028A150A12031DD02F09308A11E32201
:101FD00083160313CF01D001DC0102308A004F08C1
:101FE0008A110A126A228A110A12E3228316031343
:101FF000CF0A0319D00ADC0A04305C028A150A12DF
:10200000031DED2F09308A11E3220D308A110A12C7
:10201000E3220A308A110A12E322F03083160313F6
:10202000CF00D001DD015008D3004F082A07D200AD
:102030000318D30AF0308312A400A50183165208B6
:102040008312A000831653088312A1008A110A127A
:1020500091228312031322088316AB0083122308F4
:102060008316AC001B30AC075830AB070318AC0A22
:102070002B080317BE0003132C080317BF008A1197
:102080000A1232248312031320088316C700831216
:1020900021088316C8000310C70DC80D033048027D
:1020A0008A110A16031D5628E730470203195E28D5
:1020B000031C5E28E730C7000330C800F030AB07D0
:1020C0000318AC0A2B080317BE0003132C080317D0
:1020D000BF000A1232248312031320088316C9009A
:1020E000831221088316CA000310C90DCA0D0330DC
:1020F0004A028A110A16031D7F28E7304902031994
:102100008728031C8728E730C9000330CA00F03055
:10211000AB070318AC0A2B080317BE0003132C08E7
:102120000317BF000A1232248312031320088316F8
:10213000CB00831221088316CC000310CB0DCC0DED
:1021400003304C028A110A16031DA828E7304B02FF
:102150000319B028031CB028E730CB000330CC00B3
:10216000F030AB070318AC0A2B080317BE000313AB
:102170002C080317BF000A1232248312031320080D
:102180008316CD00831221088316CE000310CD0DD7
:10219000CE0D03304E028A110A16031DD128E730F6
:1021A0004D020319D928031CD928E730CD0003308C
:1021B000CE00E8308312A4000330A50083164F0838
:1021C0008312A000831650088312A1000A129122E4
:1021D0008312031322088316D20083122308831666
:1021E000D30064308312A400A50183165208831221
:1021F000A000831653088312A1008A110A129122AB
:102200008312031326088316D4008312270883162B
:10221000D5005508D70030305407D6000318D70A28
:1022200056088A110A12E322643083120313A400B1
:10223000A50183164F088312A0008316500883124D
:10224000A1008A110A129122831203132208831615
:10225000D200831223088316D3000A308312A4000D
:10226000A501831652088312A00083165308831217
:10227000A1008A110A1291228312031326088316E1
:10228000D400831227088316D5005508D7003030B4
:102290005407D6000318D70A56088A110A12E322F7
:1022A0000A3083120313A400A50183164F0883127A
:1022B000A000831650088312A1008A110A129122ED
:1022C0008312031322088316D20083122308831675
:1022D000D3005308D50030305207D4000318D50A74
:1022E00054088A110A12E32209308A110A12E322E1
:1022F0002D308A110A12E322E83083120313A4005E
:102300000330A500831647088312A00083164808EF
:102310008312A1008A110A12912283120313220848
:102320008316D200831223088316D30064308312ED
:10233000A400A501831652088312A0008316530837
:102340008312A1008A110A12912283120313260814
:102350008316D400831227088316D5005508D700AA
:1023600030305407D6000318D70A56088A110A12CB
:10237000E3222C308A110A12E32264308312031301
:10238000A400A501831647088312A00083164808FD
:102390008312A1008A110A129122831203132208C8
:1023A0008316D200831223088316D3000A308312C7
:1023B000A400A501831652088312A00083165308B7
:1023C0008312A1008A110A12912283120313260894
:1023D0008316D400831227088316D5005508D7002A
:1023E00030305407D6000318D70A56088A110A124B
:1023F000E3220A3083120313A400A50183164708C1
:102400008312A000831648088312A1008A110A12C1
:1024100091228312031322088316D2008312230809
:102420008316D3005308D50030305207D400031868
:10243000D50A54088A110A12E32209308A110A12B5
:10244000E3222D308A110A12E322E83083120313AB
:10245000A4000330A500831649088312A000831648
:102460004A088312A1008A110A12912283120313CF
:1024700022088316D200831223088316D300643007
:102480008312A400A501831652088312A0008316AC
:1024900053088312A1008A110A1291228312031396
:1024A00026088316D400831227088316D500550802
:1024B000D70030305407D6000318D70A56088A11BF
:1024C0000A12E3222C308A110A12E32264308312AA
:1024D0000313A400A501831649088312A0008316E4
:1024E0004A088312A1008A110A129122831203134F
:1024F00022088316D200831223088316D3000A30E1
:102500008312A400A501831652088312A00083162B
:1025100053088312A1008A110A1291228312031315
:1025200026088316D400831227088316D500550881
:10253000D70030305407D6000318D70A56088A113E
:102540000A12E3220A3083120313A400A5018316A2
:1025500049088312A00083164A088312A1008A1139
:102560000A1291228312031322088316D2008312C7
:1025700023088316D3005308D50030305207D40007
:102580000318D50A54088A110A12E32209308A1165
:102590000A12E322E83083120313A4000330A500DB
:1025A00083164B088312A00083164C088312A100E7
:1025B0008A110A1291228312031322088316D20071
:1025C000831223088316D30064308312A400A5016C
:1025D000831652088312A000831653088312A100A9
:1025E0008A110A1291228312031326088316D4003B
:1025F000831227088316D5005508D70030305407BA
:10260000D6000318D70A56088A110A12E3222C3082
:102610008A110A12E322643083120313A400A50175
:1026200083164B088312A00083164C088312A10066
:102630008A110A1291228312031322088316D200F0
:10264000831223088316D3000A308312A400A50145
:10265000831652088312A000831653088312A10028
:102660008A110A1291228312031326088316D400BA
:10267000831227088316D5005508D7003030540739
:10268000D6000318D70A56088A110A12E3220A3024
:1026900083120313A400A50183164B088312A00024
:1026A00083164C088312A1008A110A129122831208
:1026B000031322088316D200831223088316D30043
:1026C0005308D50030305207D4000318D50A5408F7
:1026D0008A110A12E32209308A110A12E322E83031
:1026E00083120313A4000330A50083164D08831240
:1026F000A00083164E088312A1008A110A129122AB
:102700008312031322088316D20083122308831630
:10271000D30064308312A400A501831652088312EB
:10272000A000831653088312A1008A110A12912275
:102730008312031326088316D400831227088316F6
:10274000D5005508D70030305407D6000318D70AF3
:1027500056088A110A12E3222C308A110A12E32247
:10276000643083120313A400A50183164D0883125D
:10277000A00083164E088312A1008A110A1291222A
:102780008312031322088316D200831223088316B0
:10279000D3000A308312A400A501831652088312C5
:1027A000A000831653088312A1008A110A129122F5
:1027B0008312031326088316D40083122708831676
:1027C000D5005508D70030305407D6000318D70A73
:1027D00056088A110A12E3220A3083120313A40056
:1027E000A50183164D088312A00083164E0883129C
:1027F000A1008A110A129122831203132208831660
:10280000D200831223088316D3005308D50030303A
:102810005207D4000318D50A54088A110A12E32279
:102820000D308A110A12E3220A308A110A12E322B9
:1028300083160313CF034F0A0319D0030A3003177B
:10284000A400A5018A110A12BE2483160313DD0A0F
:10285000F0305D028A110A16031D132808000A30A1
:1028600003179E009F010A12E8240130831203130C
:10287000D7008A150A127420023083160313BB0096
:102880000A30BC003B088312D80083163C08831230
:10289000D900543083160317930009309400183080
:1028A000950096014D3097000230403898008A110B
:1028B0000A1218250A3083160317A400A5018A11ED
:1028C0000A12BE24023083160313BD001930BE0065
:1028D0003D088312D80083163E088312D900543075
:1028E0008316031793000930940018309500960161
:1028F000343097000230403898008A110A121825A7
:102900000A3083160317A400A5018A110A12BE24F7
:10291000023083160313BF003230C0003F08831219
:10292000D800831640088312D90054308316031749
:102930009300093094001830950096011B309700E1
:102940000230403898008A110A1218251430831674
:1029500003179E009F018A110A12E82483160313AD
:10296000B201A801A90103108316280DB300290D97
:10297000B4000310280DB500290DB6003509B700C5
:102980003609B8008130B7070318B80A3808BA000A
:102990003703B900390A0319BA0383120317AB01CD
:1029A00083160313390883120317AC003F30AD00C0
:1029B0008316031333088A150A1265210A30831619
:1029C0000317A400A5018A110A12BE24831603135B
:1029D000A80A0319A90A3F3028028312A000003078
:1029E00083162902831220048A110A16031DB32CB0
:1029F0008316A801A90183162809B3002909B40088
:102A00004130B3070318B40A280883120317AB0038
:102A1000AC0183160313330883120317AD007F3014
:102A20008A150A1265210A3083160317A400A5012E
:102A30008A110A12BE2483160313A80A0319A90ACD
:102A40003F3028028312A00000308316290283122F
:102A500020048A110A16031DFB2CD7018316B20A23
:102A600002303202031DB12C0A3003179E009F0171
:102A70000A12E8248A150A127420831203138A1199
:102A80000A1605189E2D0130D70002308316C300A8
:102A90001930C40043088312D800831644088312F7
:102AA000D90054308316031793000930940019306D
:102AB00095009601D13097000130403898000A12F5
:102AC00018250A3083160317A400A5018A110A12DB
:102AD000BE24573083160313A8001B30A900C10180
:102AE000C201831628080317AA0003132908031735
:102AF000AB00FF30AC00AD018A110A1248248316E6
:102B00000313A80A0319A90AC10A0319C20ACA3081
:102B100041028312A0000330831642028312200474
:102B20008A110A16031D712D0A3083160317A4009B
:102B3000A5010A12BE248A150A1274208A150A12E7
:102B4000BF228A150A1221243A3083120313680225
:102B50008A110A160319B22D8A150A129F238A11A7
:102B60000A16A42D8A150A129F23313083120313EB
:102B700068028A110A16031DDF2E8A150A129F2386
:102B80002E308312031368028A110A16031DDF2EEA
:102B90008A150A129F2337308312031368028A11A1
:102BA0000A16031DDF2E8A150A129F232E30831268
:102BB000031368028A110A16031DDF2E8A150A12F2
:102BC0009F2330308312031368028A110A16031DF3
:102BD000DF2E8A150A129F232830831203136802FE
:102BE0008A110A16031DDF2EE9018316C5018A1515
:102BF0000A129F235A308312031369078400831338
:102C000068088000E90A8316C50A073045028A1160
:102C10000A16031DF72D28308312031368020319C7
:102C2000172E8A150A129F238A110A160B2EE90104
:102C30008316C6018A150A129F236130831203137B
:102C400069078400831368088000E90A8316C60AAE
:102C5000073046028A110A16031D1A2E30308312DD
:102C60005D028316B30033088312A000A101643013
:102C7000A200A3010A127E228312031324088316E2
:102C8000B400303083125F028316B500350883121A
:102C9000A000A1010A30A200A3018A110A127E221B
:102CA0008312031324088316B60036083407B700CE
:102CB0003030831260028316B80038083707831259
:102CC000EA00EB01303064028316B300330883124C
:102CD000A000A1016430A200A3018A110A127E2281
:102CE0008312031324088316B40030308312660263
:102CF0008316B50035088312A000A1010A30A20096
:102D0000A3018A110A127E22831203132408831658
:102D1000B60036083407B7003030831267028316D6
:102D2000B800380837078312EC00ED016B088316F2
:102D3000A10783126A088316A0070318A10A831249
:102D40006D088316A30783126C088316A207031865
:102D5000A30A8312EE0A0319EF0A831625088312C9
:102D60006B028A110A16031DB92E831624088312DA
:102D70006A020319C42E031CC42E6A088316A40019
:102D800083126B088316A5008316270883126D0231
:102D9000031DCE2E8316260883126C020319D92E2A
:102DA000031CD92E6C088316A60083126D088316A7
:102DB000A7008A150A127A258A150A12A723FE018E
:102DC000831203136F087E028A110A16031DEB2E6D
:102DD0006E08831631020319F22E0318F22E8A159B
:102DE0000A122226831203138A110A16051AA42D29
:0C2DF0008A150A1248278A110A16A42D21
:02400E004A2F37
:00000001FF
